:020000040000FA
:04000000DAEF00F043
:08000800046E7F0B04BC8008AC
:10001000F76A200FF66E0800F55004BE00081200C3
:10002000000306090C101316191C1F2225282B2E5D
:10003000313336393C3F414447494C4E5153555872
:100040005A5C5E60626466686A6B6D6F707173742F
:10005000757678797A7A7B7C7D7D7E7E7E7F7F7FE8
:100060007F00106A116A01D0086E0950085ED8A09E
:1000700009061150105ED8A01106D8900932083236
:10008000D89011321032011C066E021C076E062A2F
:10009000D8B4072A830E0B6E0C6A0D6A0E6A0F6ABB
:1000A0000A6A0F0EEA6E00C0E9FF031CB4EC00F010
:1000B00000D000D0000008500C26D8B00D2A0950FE
:1000C0000D2610500E26D8B00F2A11500F260D50B5
:1000D0009BDF800F056E0F5097DF800F05260530E0
:1000E0000A2600C0E9FFEF500310D8A00318EF6EF6
:1000F0000B04D8B4830E0B6ED8B4062AD8B4073ECE
:10010000D7D71200076A066EFF0E0626072200D018
:10011000D8A01200030E056EE70E02D8F5D7056AC7
:10012000FD0F046EFF0E00D001D00426000000D0A9
:10013000D8A00526D8A01200F8D7096A086A100EC0
:10014000F36E0534083609360650085C0750095826
:1001500005E30650085E0750095AD8800436053674
:10016000F32EEFD704501200E988E92AEC161200AA
:10017000A66AA68E0900F55002E0EE6EFBD71200CB
:10018000F34E02D0E652FCD7E6CFEEFFE82EFCD7C6
:1001900012004351204351204351204445205736FB
:1001A0004142432057364142432057364142432083
:1001B000204B0000F86AAB6A640EA4DF9498829822
:1001C000949A829A9390819093928192939481943D
:1001D0000B0EC16EF19E00EE18F0010EF76E920E3E
:1001E000F66EC6DFEF6A0F0E166E040E056EB00EC9
:1001F000046E076A16C006F0A0DF146E05C015F085
:10020000030E136E520E126E5892588058B08282AE
:1002100058A0829280AA0FEF01F010EC01F0FAD7FB
:100220009492828200EE18F0E86AEE5202E0E83E14
:10023000FCD7176E010E556E5550175CD8A06CEFA9
:1002400003F000EE4BF010EE18F055C0F3FF010E76
:1002500097DFEF6A410E4B6237EF01F000EE4FF08F
:100260002E0EEE6E2D0EEE6EEF6A66EF03F0420E6E
:100270004B6246EF01F000EE4FF02D0EEE6E2E0EAB
:10028000EE6EEE6EEE6EEF6A66EF03F0430E4B62BB
:1002900057EF01F000EE4FF02D0EEE6E2E0EEE6ECB
:1002A0002D0EEE6E2E0EEE6EEF6A66EF03F0440E2C
:1002B0004B6265EF01F000EE4FF02D0EEE6E2E0E4C
:1002C000EE6EEE6EEF6A66EF03F0450E4B6270EF76
:1002D00001F000EE4FF02E0EEE6EEF6A66EF03F0C7
:1002E000460E4B6280EF01F000EE4FF02E0EEE6EE8
:1002F000EE6E2D0EEE6E2E0EEE6EEF6A66EF03F0D2
:10030000470E4B628EEF01F000EE4FF02D0EEE6EB9
:10031000EE6E2E0EEE6EEF6A66EF03F0480E4B6245
:100320009CEF01F000EE4FF02E0EEE6EEE6EEE6ED4
:10033000EE6EEF6A66EF03F0490E4B62A8EF01F034
:1003400000EE4FF02E0EEE6EEE6EEF6A66EF03F0EB
:100350004A0E4B62B7EF01F000EE4FF02E0EEE6E3C
:100360002D0EEE6EEE6EEE6EEF6A66EF03F04B0E44
:100370004B62C6EF01F000EE4FF02D0EEE6E2E0E2A
:10038000EE6E2D0EEE6EEF6A66EF03F04C0E4B62D2
:10039000D6EF01F000EE4FF02E0EEE6E2D0EEE6E4B
:1003A0002E0EEE6EEE6EEF6A66EF03F04D0E4B62B0
:1003B000E2EF01F000EE4FF02D0EEE6EEE6EEF6A02
:1003C00066EF03F04E0E4B62EFEF01F000EE4FF0E0
:1003D0002D0EEE6E2E0EEE6EEF6A66EF03F04F0EF0
:1003E0004B62FCEF01F000EE4FF02D0EEE6EEE6E64
:1003F000EE6EEF6A66EF03F0500E4B620CEF02F008
:1004000000EE4FF02E0EEE6E2D0EEE6EEE6E2E0EF8
:10041000EE6EEF6A66EF03F0510E4B621CEF02F0D6
:1004200000EE4FF02D0EEE6EEE6E2E0EEE6E2D0ED9
:10043000EE6EEF6A66EF03F0520E4B622BEF02F0A6
:1004400000EE4FF02E0EEE6E2D0EEE6E2E0EEE6EB8
:10045000EF6A66EF03F0530E4B6238EF02F000EEE6
:100460004FF02E0EEE6EEE6EEE6EEF6A66EF03F05C
:10047000540E4B6243EF02F000EE4FF02D0EEE6E85
:10048000EF6A66EF03F0550E4B6251EF02F000EE9B
:100490004FF02E0EEE6EEE6E2D0EEE6EEF6A66EFE4
:1004A00003F0560E4B6260EF02F000EE4FF02E0E9E
:1004B000EE6EEE6EEE6E2D0EEE6EEF6A66EF03F0F0
:1004C000570E4B626EEF02F000EE4FF02E0EEE6E06
:1004D0002D0EEE6EEE6EEF6A66EF03F0580E4B6275
:1004E0007EEF02F000EE4FF02D0EEE6E2E0EEE6E51
:1004F000EE6E2D0EEE6EEF6A66EF03F0590E4B6254
:100500008EEF02F000EE4FF02D0EEE6E2E0EEE6E20
:100510002D0EEE6EEE6EEF6A66EF03F05A0E4B6232
:100520009DEF02F000EE4FF02D0EEE6EEE6E2E0EF1
:10053000EE6EEE6EEF6A66EF03F0300E4B62ACEFDC
:1005400002F000EE4FF02D0EEE6EEE6EEE6EEE6EE1
:10055000EE6EEF6A66EF03F0310E4B62BCEF02F015
:1005600000EE4FF02E0EEE6E2D0EEE6EEE6EEE6E77
:10057000EE6EEF6A66EF03F0320E4B62CCEF02F0E4
:1005800000EE4FF02E0EEE6EEE6E2D0EEE6EEE6E57
:10059000EE6EEF6A66EF03F0330E4B62DCEF02F0B3
:1005A00000EE4FF02E0EEE6EEE6EEE6E2D0EEE6E37
:1005B000EE6EEF6A66EF03F0340E4B62EBEF02F083
:1005C00000EE4FF02E0EEE6EEE6EEE6E2D0EEE6E17
:1005D000EF6A66EF03F0350E4B62FAEF02F000EEC1
:1005E0004FF02E0EEE6EEE6EEE6EEE6EEE6EEF6A6B
:1005F00066EF03F0360E4B620AEF03F000EE4FF0A9
:100600002D0EEE6E2E0EEE6EEE6EEE6EEE6EEF6A4E
:1006100066EF03F0370E4B621AEF03F000EE4FF077
:100620002D0EEE6EEE6E2E0EEE6EEE6EEE6EEF6A2E
:1006300066EF03F0380E4B622AEF03F000EE4FF046
:100640002D0EEE6EEE6EEE6E2E0EEE6EEE6EEF6A0E
:1006500066EF03F0390E4B623AEF03F000EE4FF015
:100660002D0EEE6EEE6EEE6EEE6E2E0EEE6EEF6AEE
:1006700066EF03F02F0E4B624CEF03F000EE4FF0ED
:100680002D0EEE6E2E0EEE6EEE6E2D0EEE6E2E0E0C
:10069000EE6EEF6A66EF03F03D0E4B625DEF03F026
:1006A00000EE4FF02D0EEE6E2E0EEE6EEE6EEE6E36
:1006B0002D0EEE6EEF6A66EF03F0200E4B6266EFD2
:1006C00003F000EE4FF0200EEE6EEF6A6DEC03F0DB
:1006D000552AD8A41CEF01F0120000EE4FF0E86A92
:1006E000EE5202E0E83EFCD7566E010E576E5750B0
:1006F000565CD8A0D4EF03F000EE4DF010EE4FF0B2
:1007000057C0F3FF010EC0EC00F0EF6A2E0E4D62F1
:100710009EEF03F093948184820E006E040E036EAC
:1007200015C002F014C001F013C009F012C008F0A7
:1007300031EC00F093948194CCEF03F02D0E4D62D8
:10074000BCEF03F093948184820E006E040E036E5E
:100750001550030DF3CF02F01450030DF3CF01F049
:10076000F450022613C009F012C008F031EC00F07A
:1007700093948194CCEF03F0200E4D62CCEF03F004
:100780001550030DF3CF07F01450030DF3CF06F00F
:10079000F450072684EC00F015C007F0145083ECE9
:1007A00000F0572AD8A4A3D71550030DF3CF07F0B4
:1007B0001450030DF3CF06F0F450072684EC00F03C
:0207C000120025
:020000040030CA
:03000100861A0F4D
:020005008181F7
:060008000FC00FE00F40E5
:00000001FF
